:020000040000FA
:1000000010284E34413456344C3436343734353479
:100010002D342D34563430342E3433342D342D34A5
:100020002010031E20148316FF23900083128316D2
:1000300087308100831200308500831608308500E8
:100040009F0183120730990051288A0123088207F3
:1000500001340034013400340134003400340034FD
:100060000034003400340034003480348A01240821
:10007000820700340034003400340034013400348A
:100080000134003401340034003400348034A600DC
:10009000C730A70064000000A70B4A28A60B482819
:1000A000003420186128A001FA304720373085003D
:1000B000FA304720003085000430A200A301A401DB
:1000C000A50181016400811BB32885196228810183
:1000D0006400811BB328851D6828A1016400A10A62
:1000E0000319AD287328000085196E2846302102B7
:1000F000031CAD28A01182302102031CA015AA30D8
:100100002102031C862800308500A82885140514C8
:10011000A01D0511A0190515A20BA8280430A200E6
:100120002520A600A30AA61BA301A0102618A01430
:100130003620A600A40AA61BA4012011261820150B
:10014000A0188516A01C851220190516201D051261
:10015000A5080319B528A503B528A50A0A30250264
:0C016000031CB528A503003085006128B1
:0207FE00903435
:02400E00DC3F95
:00000001FF
